:020000020000FC
:1000000012C0E2C01895189518951895189518956E
:100010001895189518951895189518951895189578
:100020001895189518954CEA4DBFBB27DD27FF277B
:10003000112442E0142AEE2417D228D2EED19CD10A
:1000400040E048BB40EF42BB40E041BB44274FBBD0
:100050004EE946B940EC47B943E945BF40E44BBFE0
:10006000939A8B9A000000007894809B07C002301E
:1000700079F0033051F010FC13C0F7CF4FEF8099A7
:10008000F4CF4A95E1F778D1F0CFC2D304E0EDCFB9
:10009000C0E66C2D11D294D21FD206D304E0E5CF76
:1000A000412D4FEF4D7F4E7F142214FC3EC041E0A6
:1000B0004093B40040EC47B90000889544B14093A8
:1000C000B900389A45B1889534B125B1331F221F44
:1000D000331F221F432B4093BA00B89A2F6040B3BE
:1000E000B8983FEF4327407F4295EEE5E40F349107
:1000F000232B399A3D9A2093BB00889545B13898B7
:1001000040584093B600889544EE47B945B14058F1
:100110004093B500889545B1389A4093B7008895CB
:1001200045B14093B80018E02AC042E04093B400C3
:10013000B99A000040B3B9984F604295BA9A00004E
:1001400030B3BA983F6043274093B500BB9A000094
:1001500040B3BB984F604295BC9A000030B3BC9846
:100160003F6043274093B600BD9A000040B3BD985E
:100170004F6042953FEF43274093B70014E040E1C2
:1001800014264BEC4F9340E04F93C2EB62E0610FBB
:10019000CF936F932AC2639563954D2D4093AF0023
:1001A000482D4093AE009394C2EB96D1992460936E
:1001B000B1008092B0004091AF00D42E4091AE00CB
:1001C000842E42E0142A51CF5FB64F933F9343E011
:1001D00032E0809BFECF819BFECF819B05C043E038
:1001E0003A95000099F0F9CF32E04A950000A9F75E
:1001F00007C06F90AF911F912F91CF916F91522DAA
:100200003F914F915FBE80E48ABF1895252E80B341
:100210006F93CF9356E06EE0CEE670B37370A1F0AB
:100220007795881F5A95C9F7000070B3737061F015
:100230007795881F57E0899380B3837029F05A958A
:1002400000006A9551F7D9CFC137B8F240916E00DE
:1002500030916F0071F43E7F3F1559F4423711F42D
:1002600091E0CBCF403511F493E0C7CF4E3409F481
:100270000AC0483211F0463321F4913001F1933035
:1002800031F190E0BACF2F931F93AF936F923091DB
:100290006F002091700037952795229530FF01C09F
:1002A00020952F702A3019F02530E9F0A2CF0430C4
:1002B000B9F46CD0EE20B1F492E003E09ACF2F9322
:1002C0001F93AF936F92D7D040D002E092CF2F937D
:1002D0001F93AF936F92023019F0CDD0002789CFD2
:1002E000DCD087CF22C011FE1FC04D2D4093AF0040
:1002F000482D4093AE004091B000842E6091B10033
:10030000C2EB46D04091AF00D42E4091AE00842E77
:100310004091B300433C11F043EC01C04BE44093E7
:10032000B30041E0142A65CF64CFFF2421E018E038
:100330004F2DE79408F042274795FF1C1A95C1F707
:10034000EE242F2D2E7FF22E54CF573029F05395C7
:10035000881F5A95E9F789936C2F6D56C62ECEE605
:10036000A1E6BF93BB2749914D936A95E1F7BF91F1
:1003700064E56093600008954AEAF42E9927992471
:100380008824002733243092C80008956D2DCFECC7
:1003900030E0162F23E079919198909A899A889A63
:1003A00042B357E00000779508F0422742BB5A95C8
:1003B000C9F770FF42271A95799142BB91F7582DE2
:1003C000503041F0779508F0422742BB00005A9523
:1003D000C9F7788100004C7F42BB55E05A95F1F790
:1003E000909A909A89988898909808954091D00012
:1003F0004B3443EC09F04BE44093D000089543ECB8
:100400004093D00040E84093CF00F0DF40E04093BD
:10041000D1004093D20064E0089548E0A42E40E863
:100420004093CF0043EC4093D0001A2D6A2DC1EDCC
:10043000C895099231966A95D9F762E0610FD2D0DA
:10044000639563959394CFEC47D0D62E9924D092A0
:10045000B1008092B0006D2DFF27EFECC2EB019050
:1004600009926A95E1F7089540E84093CC0042ED87
:100470004093CD000895CF935F938F92CCEC62E0D0
:10048000882486DF8F905F91CF91089540E8409354
:10049000C9004AE54093CA0008958F92C9EC62E012
:1004A000882476DF8F90089540E84093CF004EE196
:1004B0004093D00062E00895CF936F936C0F4FEF9D
:1004C00047954881242F2795242720952993C617DF
:1004D000B9F76F91CF910895112777247A94CF932C
:1004E0006F93312F48E0340F6A95E9F726E06F915A
:1004F0006F936C0F63956395488158E0479508F0BA
:1005000027E02A95A1F4371526E088F43A95732E52
:10051000513011F459E0C3955A9590FA1EF037D036
:100520001A9502C01BD013956F91CF91D8CF3A95F1
:1005300021F05A9519F7C395DFCF6F91CF9190FABB
:100540003EF0103051F06A95185F38F46A950895BE
:10055000812E185010F06395812E0895452F59E093
:10056000541B3881331F2FEF220F5A95E9F732239E
:100570002095269548814223342B4881441F399386
:10058000C61301C008953881331F3993F9CF452F21
:1005900059E0541B4C2F4395C62F3A913795388319
:1005A000C413FBCF3A9137952FEF5A9511F0220FD4
:1005B000FCCF3223209548814223342B3883089581
:1005C000CF936F93C0E603D06F91CF9108956C0FD6
:1005D000488138E04795221F3A95E1F72993C617DD
:1005E000B9F70895CF936F93CFEC0AD0409530952B
:1005F00039934883CA9562E0EADF6F91CF910895FD
:100600006C0FC3954991433C11F04B34A9F44FEF63
:100610003FEF299118E037FB50F95227441F331F51
:100620004E7F2695579520F450E8352755E045270D
:100630001A9589F7C61769F70895C89509923196F2
:100640006A95D9F72CC0C895099233FA36F43196D9
:10065000C8950992E89433F802C0002409923196B3
:10066000625089F71CC00080099231966A95D9F7CB
:1006700016C0EEBBFFBBE09A0DB2099231966A95A7
:10068000C1F70DC040E84093CF0068E0C1ED3320D2
:1006900009F4D3CF32FCD7CF30FCE5CFEACF37FC1B
:1006A0003324A4DEC0ED089506D09394CFEC14DF7C
:1006B000D62E99240895332440916200309163002E
:1006C000407609F41BC04034B1F0403209F013C049
:1006D000313059F0323051F0333049F0393041F097
:1006E0003A3039F03B3031F091C090C08FC08EC0AD
:1006F0008DC08CC08BC08AC041E020C03030E9F092
:100700003130D1F03330C1F0353079F0363029F165
:10071000373009F13830A9F0393051F03A30B9F0BA
:100720003B3051F03C30B9F071C0E09064006EC0D5
:10073000409164004093C80069C042E0F8E0E4E7FB
:1007400052C04091C80041E0F8E0E7E54CC0F8E055
:10075000EEE541E048C0A8DE0895409162004138CE
:1007600049F030916500313071F0323081F0333032
:10077000D9F0089530916500313269F0323279F064
:10078000333289F00895F8E0E0E442E12CC0F8E06B
:10079000E2E542E228C0F8E0E4E649E024C0F8E0FF
:1007A000E6E74BE620C01FC03CE0332E30916400EA
:1007B0003030A1F0323051F0333061F0313011F08F
:1007C000BBCF24C0F8E0E6EE4EE90DC0F9E0E6E369
:1007D0004AE009C0F9E0ECE342E405C03324F8E064
:1007E000E2EE44E000C0A0906800A41608F0A42E39
:1007F0004A2DBB24477009F0B3944A2D469546957F
:100800004695B40E43EC4093D0000BC0F8DD08953C
:1008100002D04BDF08954B2D413011F4F3DD0895E4
:10082000BA943A2D385018E018F41A2DBB24B3941A
:10083000A32E28DF62E0610FD5DE639563950895EE
:1008400012010001000000087707010011000102F9
:100850000001090222000101028050090400000188
:1008600003000003092101010001226B000705813B
:100870000308000A0000050115000904A101050292
:10088000850109BA09BB1581257F7508950281028A
:1008900005010901A10009360937150025FF750872
:1008A0009502810209300931750A9502810215000D
:1008B00026FF03C009393500463B011601FE15002D
:1008C0002507651475049501814285020509190102
:1008D000291815002501750195185500650081023C
:1008E000C000040309009E034D696E646175676171
:1008F00073204D696C61736175736B617320262081
:100900004C617A7943616D656C202863292032300F
:1009100030342C20496E672E2049676F7220436562
:10092000736B6F2C20436F707972696768742863EA
:100930002920323030330A034D4A6F7942034D4A41
:100940006F792C2041544D65676138206261736571
:100950006420555342204A6F79737469636BF000C9
:0E096000201040F030F06070F0F050F0F0F039
:00000001FF
